:100000000C9463000C948B000C948B000C948B006C
:100010000C948B000C948B000C948B000C94270890
:100020000C948B000C948B000C948B000C948B0024
:100030000C948B000C948B000C948B000C948B0014
:100040000C94DD070C948B000C94AB070C94850783
:100050000C948B000C948B000C948B000C948B00F4
:100060000C948B000C948B000000000023002600F1
:10007000290000000000240027002A0000000000E2
:10008000250028002B0004040404040404040202D4
:100090000202020203030303030301020408102007
:1000A0004080010204081020010204081020000012
:1000B0000008000201000003040700000000000027
:1000C0000000E708231311241FBECFEFD8E0DEBFE6
:1000D000CDBF23E0AAE6B1E001C01D92A335B2076F
:1000E000E1F711E0A0E0B1E0E6ECF4E302C0059036
:1000F0000D92AA36B107D9F710E0C2E6D0E004C0ED
:100100002197FE010E945715C136D107C9F70E94F9
:10011000B5090C94561A0C9400000895AF92BF9242
:10012000CF92DF92EF92FF920F931F93CF93DF93C3
:100130006C017B018B01040F151FEB015E01AE18F2
:10014000BF08C017D10759F06991D601ED91FC9114
:100150000190F081E02DC6010995892B79F7C50141
:10016000DF91CF911F910F91FF90EF90DF90CF9093
:10017000BF90AF900895FC01538D448D252F30E042
:10018000842F90E0821B930B541710F0CF960895A4
:1001900001970895FC01918D828D981761F0A28DD1
:1001A000AE0FBF2FB11D5D968C91928D9F5F9F7397
:1001B000928F90E008958FEF9FEF0895FC01918D4D
:1001C000828D981731F0828DE80FF11D858D90E0BA
:1001D00008958FEF9FEF0895FC01918D228D892F57
:1001E00090E0805C9F4F821B91098F73992708953F
:1001F0008AEB91E00E94EC0021E0892B09F420E0D9
:10020000822F0895FC01A48DA80FB92FB11DA35A08
:10021000BF4F2C91848D90E001968F739927848F26
:10022000A689B7892C93A089B1898C918370806449
:100230008C93938D848D981306C00288F389E02DEA
:1002400080818F7D80830895EF92FF920F931F939B
:10025000CF93DF93EC0181E0888F9B8D8C8D981379
:100260001AC0E889F989808185FF15C09FB7F89485
:10027000EE89FF896083E889F989808183708064D1
:1002800080839FBF81E090E0DF91CF911F910F911C
:10029000FF90EF900895F62E0B8D10E00F5F1F4F2B
:1002A0000F731127E02E8C8D8E110CC00FB607FC3A
:1002B000FACFE889F989808185FFF5CFCE010E94C8
:1002C0000201F1CFEB8DEC0FFD2FF11DE35AFF4F33
:1002D000F0829FB7F8940B8FEA89FB898081806256
:1002E000CFCFCF93DF93EC01888D8823B9F0AA8913
:1002F000BB89E889F9898C9185FD03C0808186FDE1
:100300000DC00FB607FCF7CF8C9185FFF2CF80812F
:1003100085FFEDCFCE010E940201E9CFDF91CF91A1
:100320000895833081F028F4813099F08230A9F06B
:1003300008958730A9F08830C9F08430B1F48091F5
:1003400080008F7D03C0809180008F778093800034
:10035000089584B58F7784BD089584B58F7DFBCFD4
:100360008091B0008F778093B00008958091B000A5
:100370008F7DF9CF1F93CF93DF93282F30E0F901C2
:10038000E255FF4F8491F901E656FF4FD491F901F0
:10039000EA57FF4FC491CC23A9F0162F81110E9478
:1003A0009101EC2FF0E0EE0FFF1FE458FF4FA591F5
:1003B000B4918FB7F894EC91111108C0D095DE2359
:1003C000DC938FBFDF91CF911F910895DE2BF8CF83
:1003D000CF93DF93EC0180913D0390913E03029710
:1003E00049F4C130D10509F43BC06CF560E02097B9
:1003F00009F437C080913D0390913E03049749F47E
:10040000C130D10509F45CC00CF037C0209709F465
:1004100042C080913D0390913E03059709F0E5C0ED
:10042000CA30D10508F0E1C0FE01E75EFD4F0C9433
:100430005715780284029502AB02C602C802CF02A9
:10044000DB02EC02F302C230D105A9F060E0C33058
:10045000D10581F6809141030E94BA0160E006C097
:1004600061E0809141030E94BA0161E08091430301
:100470000E94BA01BFCF61E0EDCFC230D10539F1A2
:10048000C330D10509F0C5CF61E0809141030E94DE
:10049000BA0160E022C061E0809141030E94BA018C
:1004A00060E0809143030E94BA0161E080914503BE
:1004B0000E94BA0160E0809147030E94BA01A9CF6F
:1004C00060E0809141030E94BA0161E0EACF60E000
:1004D000809141030E94BA0161E0809143030E9430
:1004E000BA0160E0809145030E94BA0161E0E3CF68
:1004F00060E0809141030E94BA0161E08091430372
:100500000E94BA0161E00BC060E0809141030E944B
:10051000BA0161E0809143030E94BA0160E08091DA
:1005200045030E94BA0160E010C060E08091410381
:100530000E94BA0161E0809143030E94BA0160E029
:10054000809145030E94BA0161E0809147030E94B7
:10055000BA0161E015C060E0809141030E94BA01D8
:1005600061E0809143030E94BA0160E080914503FD
:100570000E94BA0161E0809147030E94BA0160E0E5
:1005800080914903DF91CF910C94BA0161E0E4CFEF
:1005900061E0809141030E94BA0160E0E2CF61E036
:1005A000809141030E94BA0160E0809143030E9460
:1005B000BA0161E0DBCF61E0809141030E94BA01A2
:1005C00060E0809143030E94BA0161E0809145039D
:1005D0000E94BA0160E0CFCF61E0809141030E94A8
:1005E000BA0160E08BCF60E0F8CFDF91CF91089542
:1005F000CF93DF9390E0FC01E656FF4F24918A579A
:100600009F4FFC0184918823D1F090E0880F991FBF
:10061000FC01EE58FF4FA591B491FC01E458FF4F47
:10062000C591D49161110EC09FB7F8948C91E22FBF
:10063000E0958E238C932881E223E8839FBFDF918E
:10064000CF9108958FB7F894EC91E22BEC938FBF84
:10065000F6CFCF93DF93EC0161E085E00E94F802D2
:10066000209731F460E085E0DF91CF910C94BA01DE
:10067000CF3FD10511F461E0F6CFE3EBF0E0E49178
:10068000E33029F140F4E130B1F0E230D9F0C03884
:10069000D1058CF7E7CFE73021F1E83051F1E430B4
:1006A000B1F780918000806280938000D0938B00AE
:1006B000C0938A0004C084B5806884BDC7BDDF9143
:1006C000CF91089584B5806284BDC8BDF8CF809174
:1006D0008000806880938000D0938900C093880058
:1006E000EECF8091B00080688093B000C093B300DB
:1006F000E6CF8091B00080628093B000C093B400D8
:10070000DECF3FB7F89480916F0190917001A09176
:100710007101B091720126B5A89B05C02F3F19F059
:100720000196A11DB11D3FBFBA2FA92F982F882771
:10073000BC01CD01620F711D811D911D42E0660F4C
:10074000771F881F991F4A95D1F708954F925F929E
:100750006F927F928F929F92AF92BF92EF92FF9291
:100760000F931F93CF93DF93EC0197FF04C0CC2727
:10077000DD27C81BD90B181619060CF061C081E0E3
:1007800090E0909336038093350304E010E08AE014
:10079000E82EF12C209709F46FC00E94810380900D
:1007A0004B0390904C03A0904D03B0904E032B014F
:1007B0003C01481859086A087B08809037039090DC
:1007C0003803A0903903B0903A03481459046A04DE
:1007D0007B0400F360934B0370934C0380934D03B1
:1007E00090934E0380913F039091400320913503F5
:1007F000309136032130310559F50196909340032D
:1008000080933F0320913B0330913C038217930771
:1008100021F41092400310923F03219780913F03EF
:100820009091400320913D0330913E03B701253064
:10083000310509F0B8010E9424150E94E801AACFF1
:10084000892B09F4A2CF10923603109235039DCF65
:10085000892B41F480913B0390913C03909340039A
:1008600080933F0380913F039091400301979093C1
:10087000400380933F03D1CFDF91CF911F910F9120
:10088000FF90EF90BF90AF909F908F907F906F9070
:100890005F904F9008958F929F92AF92BF92CF92A8
:1008A000DF92EF92FF926B017C010E9481034B016A
:1008B0005C01C114D104E104F104B9F00E94810388
:1008C000681979098A099B09683E73408105910579
:1008D00080F321E0C21AD108E108F10888EE880E01
:1008E00083E0981EA11CB11CE4CFFF90EF90DF9035
:1008F000CF90BF90AF909F908F9008952FB7F894AE
:1009000060916B0170916C0180916D0190916E010D
:100910002FBF0895CF92DF92EF92FF920F931F9314
:10092000CF93DF93442331F18C01D0E0C0E06B0121
:10093000770FEE08FF0861E081E10E94BA01C7016C
:10094000B6010E944B0460E081E10E94BA0162E3BB
:1009500070E080E090E00E944B0421960C171D0788
:1009600051F7DF91CF911F910F91FF90EF90DF90A2
:10097000CF9008956E5C7F4F072E000C880B990B6B
:10098000DF91CF911F910F91FF90EF90DF90CF906B
:100990000C944B0460E086E00E94BA0160E087E0BE
:1009A0000E94BA0160E088E00E94BA0160E089E03C
:1009B0000C94BA01EF92FF920F931F93CF93DF93A2
:1009C0007C010AE911E0D0E0C0E0F80161918F01FB
:1009D000C7018C0F9D1F0E94B5142196C032D1050E
:1009E000A1F780E290E0DF91CF911F910F91FF90EE
:1009F000EF90089580917801909179010C94DA0438
:100A0000CF93DF93EC0181E090E09093B10180936C
:100A1000B00110929F0110929E010E94FA04CE0133
:100A20000E94A6038091B2019091B301009739F41E
:100A300082E090E090939F0180939E0103C08130FB
:100A40009105C1F31092B1011092B00182E090E0E3
:100A50009093B3018093B2010E94FA04DF91CF9189
:100A60000C94CA040F931F93CF93DF93CAE9D1E08C
:100A70008C010A591140C8018C0F9D1F0E94AD14B2
:100A8000899381E0CA3BD807B1F780E290E0DF911B
:100A9000CF911F910F910895FC0180819181009762
:100AA00011F00C944D1360E070E0CB0108950F93AA
:100AB0001F93CF93DF938C01EB01FC018081918127
:100AC0000097E1F06881798161157105A9F0428193
:100AD00053812C813D814217530770F00E947E178D
:100AE0008C819D81F801958384831D821C82DF9116
:100AF000CF911F910F9108950E942F16888199819F
:100B0000F801918380838A819B81938382838C8186
:100B10009D8195838483198218821B821A82E5CF76
:100B2000CF93DF93EC0188819981009711F00E94A7
:100B30002F16198218821D821C821B821A82DF9155
:100B4000CF910895FC0180819181009711F00C9460
:100B50002F1608950F931F93CF93DF93EC01888195
:100B60009981009759F02A813B812617370730F089
:100B700081E0DF91CF911F910F9108958B016F5FFD
:100B80007F4F0E94B816009759F0998388831B8382
:100B90000A832C813D81232B59F7FC011082E8CF79
:100BA00080E0E7CFEF92FF920F931F93CF93DF93F5
:100BB000EC01FB01E080F180E114F10411F104810A
:100BC000158101151105A9F08C819D81080F191F50
:100BD000B801CE010E94AA05882399F028813981A5
:100BE0008C819D81B701820F931F0E947E171D8308
:100BF0000C83CE01DF91CF911F910F91FF90EF9069
:100C00000895CE010E949005F4CFEF92FF920F93CA
:100C10001F93CF93DF93EC017B018A01BA010E94FD
:100C2000AA0581110BC0CE010E949005CE01DF9173
:100C3000CF911F910F91FF90EF9008951D830C832A
:100C4000B701888199810E947E17F0CFFC01118243
:100C50001082138212821582148250E040E06CE30D
:100C600071E00C940506FB0101900020E9F7319733
:100C7000AF01461B570B0C940506CF93DF9300D0B2
:100C8000CDB7DEB7FC011182108213821282158269
:100C9000148269831A82BE016F5F7F4F0E94330600
:100CA0000F900F90DF91CF910895CF93DF93EC01D8
:100CB000FB018617970749F0608171816115710505
:100CC00041F0448155810E940506CE01DF91CF910C
:100CD00008950E949005F9CFFF920F931F93CF9331
:100CE000DF9300D0CDB7DEB786E0F82E8AEB91E037
:100CF0000E94EC00892B09F476C08AEB91E00E94F7
:100D0000CA00833251F08E3309F049C06CE371E0C0
:100D10008FE293E00E943306E9CF209129033091BE
:100D20002A0380912D0390912E0328173907F4F69A
:100D300040912B0350912C032091270330912803DD
:100D4000C90101969093280380932703F29EC00166
:100D5000F39E900D11246FE273E0840F951F0E94A3
:100D600055068091290390912A03019690932A03B6
:100D700080932903809127039091280320912D03CC
:100D800030912E03281739070CF0B0CF2F5F3F4F5B
:100D9000821B930B9093280380932703A7CF89830B
:100DA0001A8200913303109134030F5F1F4FB80173
:100DB0008FE293E00E94AA05882309F497CF20913F
:100DC0002F03309130038091330390913403BE019F
:100DD0006F5F7F4F820F931F0E947E171093340323
:100DE0000093330383CF0F900F90DF91CF911F912A
:100DF0000F91FF9008950E94F80081110C946C06E9
:100E000008950F931F93CF93DF93CDB7DEB7A097CD
:100E10000FB6F894DEBF0FBECDBF1F9293E29F9333
:100E20007F936F93282F082E000C330B3F938F93E3
:100E30008DE291E09F938F931F9280E28F938E01BA
:100E40000F5F1F4F1F930F930E948517F8010190AA
:100E50000020E9F73197AF01401B510BB8018AEB35
:100E600091E00E948E000FB6F894DEBF0FBECDBF9A
:100E7000A0960FB6F894DEBF0FBECDBFDF91CF9125
:100E80001F910F9108950F931F93CF93DF93CDB7C9
:100E9000DEB7A0970FB6F894DEBF0FBECDBF1F928E
:100EA00093E29F937F936F93282F082E000C330BB0
:100EB0003F938F9385E391E09F938F931F9280E2FE
:100EC0008F938E010F5F1F4F1F930F930E94851703
:100ED000F80101900020E9F73197AF01401B510B59
:100EE000B8018AEB91E00E948E000FB6F894DEBF45
:100EF0000FBECDBFA0960FB6F894DEBF0FBECDBF1C
:100F0000DF91CF911F910F9108951F920F920FB60D
:100F10000F9211242F933F934F935F936F937F937F
:100F20008F939F93AF93BF93EF93FF938AEB91E0DF
:100F30000E940201FF91EF91BF91AF919F918F911C
:100F40007F916F915F914F913F912F910F900FBEC5
:100F50000F901F9018951F920F920FB60F921124A9
:100F60002F938F939F93EF93FF93E091CA01F0919A
:100F7000CB018081E091D001F091D10182FD1BC0B5
:100F800090818091D3018F5F8F732091D40182175C
:100F900041F0E091D301F0E0E654FE4F958F80934D
:100FA000D301FF91EF919F918F912F910F900FBEE1
:100FB0000F901F9018958081F4CF1F920F920FB65B
:100FC0000F9211242F933F938F939F93AF93BF93CF
:100FD00080916B0190916C01A0916D01B0916E01B7
:100FE00030916A0123E0230F2D3758F50196A11D9A
:100FF000B11D20936A0180936B0190936C01A093C3
:101000006D01B0936E0180916F0190917001A0917C
:101010007101B09172010196A11DB11D80936F0104
:1010200090937001A0937101B0937201BF91AF9141
:101030009F918F913F912F910F900FBE0F901F9016
:10104000189526E8230F0296A11DB11DD2CF1F923D
:101050000F920FB60F9211242F933F934F935F93EC
:101060006F937F938F939F93AF93BF93CF93DF93B0
:10107000EF93FF932091570230E0F901E255FF4FC3
:101080008491F901E656FF4FD491F901EA57FF4FD9
:10109000C491CC2379F081110E949101EC2FF0E0F2
:1010A000EE0FFF1FE859FF4FA591B491EC91ED238E
:1010B00081E009F480E020915A0230915B022F5FB9
:1010C0003F4F30935B0220935A0290912403943651
:1010D00018F095E09093580290915802933009F4DB
:1010E0004CC0E0F4923011F190915902992319F01B
:1010F00081116BC02D9AFF91EF91DF91CF91BF913C
:10110000AF919F918F917F916F915F914F913F919F
:101110002F910F900FBE0F901F901895943009F4E7
:1011200048C0953009F78111DFCF09C08111DCCFAC
:1011300020915A0230915B022436310528F4109236
:101140005B0210925A02D0CF10922403E091240344
:1011500091E09E0F90932403F0E020915A02309189
:101160005B02EE0FFF1FE95AFD4F36832583109275
:101170005B0210925A0293E019C0813009F0B4CF9B
:10118000E091240391E09E0F90932403F0E02091DE
:101190005A0230915B02EE0FFF1FE95AFD4F368372
:1011A000258310925B0210925A0294E090935802A9
:1011B0009BCF882359F220915A0230915B02253649
:1011C000310508F491CF95E0F1CF2D9894CFEF92AF
:1011D000FF920F931F93CF93DF931092BD01109254
:1011E000BC0188EE93E0A0E0B0E08093BE01909354
:1011F000BF01A093C001B093C1018FE191E0909332
:10120000BB018093BA0185EC90E09093C701809375
:10121000C60184EC90E09093C9018093C80180ECF2
:1012200090E09093CB018093CA0181EC90E0909381
:10123000CD018093CC0182EC90E09093CF0180931C
:10124000CE0186EC90E09093D1018093D001109272
:10125000D3011092D4011092D5011092D6011092B0
:10126000400310923F031092360310923503109200
:101270004B0310924C0310924D0310924E0388E1E1
:1012800090E090933C0380933B0386E090E0909342
:1012900042038093410387E090E09093440380935E
:1012A000430388E090E0909346038093450389E0F0
:1012B00090E0909348038093470361E086E00E94AA
:1012C000F80261E0809143030E94F80261E080919E
:1012D00045030E94F80261E0809147030E94F802F2
:1012E00010924A031092490384E090E090933E03E9
:1012F00080933D0380935702109259028FE293E04E
:101300000E942606109226031092250310922803AD
:101310001092270310922A031092290384E190E08F
:1013200090932E0380932D0380E890E00E94931504
:10133000EC0125E130E0299339938E017C0120E80E
:10134000E20EF11CC8010E9426060A5F1F4FE0163C
:10135000F106C1F7D0932C03C0932B03DF91CF91FB
:101360001F910F91FF90EF900895CF93DF93CDB72A
:10137000DEB7C555D1090FB6F894DEBF0FBECDBF9D
:10138000789484B5826084BD84B5816084BD85B560
:10139000826085BD85B5816085BD80916E0081606C
:1013A00080936E0010928100809181008260809312
:1013B0008100809181008160809381008091800014
:1013C0008160809380008091B10084608093B1003F
:1013D0008091B00081608093B00080917A00846039
:1013E00080937A0080917A00826080937A00809165
:1013F0007A00816080937A0080917A00806880937F
:101400007A001092C100E091CA01F091CB0182E014
:101410008083E091C601F091C7011082E091C8017C
:10142000F091C9018FEC80831092D201E091CE013E
:10143000F091CF0186E08083E091CC01F091CD0165
:10144000808180618083E091CC01F091CD01808129
:1014500088608083E091CC01F091CD01808180682B
:101460008083E091CC01F091CD0180818F7D8083DC
:101470008AEB91E00E94EC00892B29F08AEB91E045
:101480000E94CA00F5CF61E081E10E94F80261E0AC
:1014900085E00E94F80261E082E00E94F80220915B
:1014A0003B0330913C03032E000C440B550B60E0D2
:1014B00077E883E993E00E943815CA01B90128EA68
:1014C00032E040E050E00E9438152093370330931B
:1014D00038034093390350933A030E94CA046CE3E3
:1014E00071E08FE293E00E9433061092790110922E
:1014F00078011092770180E290E0909376018093DA
:101500007501909374018093730110E000E0FF2453
:10151000F394C8010E94320580919A0190919B0139
:101520008336910531F41093790100937801F0929C
:101530007701005E1F4F011524E0120751F700915B
:1015400078011091790180917701882309F413C102
:10155000C8010E94320510929B0110929A01C801A5
:101560000E94DA0420917501309176018091780112
:1015700090917901820F931F909379018093780164
:101580006091730170917401269FA001279F500DF7
:10159000369F500D11248417950724F0109279017D
:1015A0001092780183E690E090939B0180939A01DA
:1015B00080917801909179010E94DA048091A401D0
:1015C000882321F061E082E00E94BA0164E670E0C5
:1015D00080E090E00E944B048091A0019091A101D5
:1015E000019709F01BC18091A2019091A3010E9473
:1015F0002903F89482E08093B0008093B10094E6D0
:101600009093B3001092B20080937000789480930E
:101610005802109224038091570260E00E94F80261
:101620004091AF0166E970E081E090E00E948A0499
:101630008E010F5F1F4F8091290390912A03181686
:1016400019060CF054C1CE01845B9F4F0E94260600
:10165000CE018A5B9F4F0E942606809129039091BC
:101660002A03009709F439C10CF0DBC0CE018E9635
:101670000E942606BE01625D7F4FCE01845B9F4FB4
:101680000E945705CE018E960E94A2056296CEACAE
:10169000DFAC6297AA24A394B12CC114D10421F029
:1016A0005601CC24C394D12CC8010E942606629610
:1016B000EEACFFAC6297CE14DF0408F5AE14BF04A5
:1016C00008F475012E96EEADFFAD2E97EE0DFF1DC1
:1016D000B08010822E966EAD7FAD2E976C0D7D1D65
:1016E000C8016115710509F4E6C00E9433062E9603
:1016F0008EAD9FAD2E97E80EF91ED701BC92B801B2
:10170000CE018A5B9F4F0E945705C8010E94A20527
:1017100062968EAD9FAD6297892B09F4DEC02E963E
:10172000EEADFFAD2E97309709F4D7C0E081E154BC
:10173000E93108F0D2C00E2E000CFF0BEE55F44F2D
:101740000C945715800E0F0EBA0DFF0DD10E910E91
:101750006D0C5E0C6D0C4A0E6D0CE90DDE0F6D0C00
:10176000900D6D0C6D0C6D0C5B0E060F6D0C820DEB
:101770006D0C160FCB0F83E690E090939B01809346
:101780009A0190939D0180939C0181E090E0909359
:101790009F0180939E011092A1011092A0011092CE
:1017A000A3011092A20121E02093A40182E090E025
:1017B0009093A6018093A50142E150E05093A801C7
:1017C0004093A70140E450E05093AA014093A9013F
:1017D00040E850E05093AC014093AB014EEF50E035
:1017E0005093AE014093AD012093AF011092B1012F
:1017F0001092B0019093B3018093B2011092B501A1
:101800001092B4018EE096E09093B7018093B601F8
:101810001092B9011092B801C801CECE90E080E0DC
:10182000E6CE209125033091260346E0429FC00179
:10183000439F900D112460912B0370912C03680F2E
:10184000791F1A8219821C821B821E821D82C80186
:101850000E9455068091250390912603019690934E
:101860002603809325032091290330912A032150D8
:10187000310930932A032093290320912D033091BD
:101880002E032817390744F42F5F3F4F821B930B19
:1018900090932603809325031FA61EA619AA18AAB3
:1018A0001BAA1AAAB801CE018E960E945705C8013C
:1018B0000E94A205DFCE0E94900519CF6BE071E077
:1018C000C8010E947E1764E670E080E090E00E940C
:1018D0004B04B80188E40E940107CE018A5B9F4F48
:1018E0000E94A205CE01845B9F4F0E94A2058CE559
:1018F00092E0909392018093910120902403312CE7
:10190000309294012092930180915802853009F021
:10191000CCC080915E0290915F02885891098D350C
:10192000910508F0C9C380912403843009F096C35F
:1019300080916002909161028097479708F08EC372
:1019400080916202909163020997099708F086C31B
:101950001092900110928F018FEF9FEFDC01809326
:101960008B0190938C01A0938D01B0938E0181E047
:1019700090E090938801809387010E947E042B0160
:101980003C0180918B0190918C01A0918D01B091CF
:101990008E018F3FEFEF9E07AE07BE0709F03BC4F5
:1019A0008091830190918401A0918501B09186017D
:1019B00080938B0190938C01A0938D01B0938E0145
:1019C00081E080938201C0908301D0908401E090F7
:1019D0008501F090860180917D01811124C0FDE395
:1019E000CF16F2ECDF06FAE9EF06F6EAFF0649F059
:1019F00027E6C21628E9D2062AE9E20626EAF20616
:101A000091F48091A0019091A101019709F09EC5E8
:101A10004091AF0164E670E081E090E00E948A04AA
:101A200081E080937D0187E6C81688E9D8068AE9B7
:101A3000E80686EAF80609F424C50CF004C4ADEF04
:101A4000CA16A2E0DA06AAE9EA06A6EAFA0609F444
:101A500042C4BDEDCB16B2E2DB06BAE9EB06B6EA4C
:101A6000FB0609F493C58091A0019091A101019713
:101A7000B9F48091A2019091A3018F3F910511F0DB
:101A8000019771F464E670E080E090E00E944B04FE
:101A90004091AF0164E670E082E090E00E948A0429
:101AA00082E0809358021092240380919901882348
:101AB00009F10E947E04C0909501D0909601E090BB
:101AC0009701F09098016C197D098E099F09693B77
:101AD0007B408105910570F00E94FA0410929901F3
:101AE0000E947E0460939501709396018093970104
:101AF000909398010E94F800882309F49CCD0E94DD
:101B00006C0696CD67E071E0C8010E947E1764E61E
:101B100070E080E090E00E944B04B80186E5DBCEE7
:101B20004091AF0168EC70E081E090E00E948A048F
:101B300080919E0190919F01029751F01092B30104
:101B40001092B2018091B6019091B7010E940005F8
:101B50004091AF0164E670E082E090E00E948A0468
:101B60006AE070E080E090E00E944B046DE371E079
:101B70008FE4B1CE4091AF0168EC70E081E090E07D
:101B80000E948A0480919E0190919F01019779F0B3
:101B900081E090E09093B3018093B2018091B6010F
:101BA0009091B7019195819591090E94000540910E
:101BB000AF0164E670E082E090E00E948A046AE08F
:101BC00070E080E090E00E944B0464E471E083E404
:101BD00082CE81E090E09093A1018093A0010E94C9
:101BE000FA048091A2019091A3010E9429036091BF
:101BF000A2017091A3018CE40E9443076ECE109263
:101C0000A1011092A0010E94FA0490E080E00E94DD
:101C1000290360919C0170919D0184E4EDCFCE0178
:101C20008A5B9F4F0E944C0597FD2EC06F3F710548
:101C30008105910509F05CF57093A3016093A20101
:101C40008091A0019091A101019719F4CB010E940C
:101C500029030E94FA048091A3018F938091A2012D
:101C60008F9386E691E09F938F931F930F930E942B
:101C7000B517B80182E40E9401070F900F900F90F2
:101C80000F900F900F9029CE70E060E0D5CF6FEFEE
:101C900070E0D2CF8091A3018F938091A2018F93A6
:101CA00086E691E09F938F931F930F930E94B51741
:101CB000B8018AE4E0CF80919F018F9380919E01CB
:101CC0008F938091A1018F938091A0018F93809138
:101CD000B1018F938091B0018F9380919D018F937B
:101CE00080919C018F938BE491E09F938F931F933E
:101CF0000F930E94B517B80183E50E9401074BC0FE
:101D00008091B9018F938091B8018F9384E591E020
:101D10009F938F931F930F930E94B517B80181E48F
:101D2000AACF1092B5011092B4011092B101109295
:101D3000B00182E090E09093B3018093B20181E022
:101D400090E090939F0180939E011092B9011092B0
:101D5000B8010E94FA048091B7018F938091B60177
:101D60008F938091B5018F938091B4018F9380E61A
:101D700091E09F938F931F930F930E94B517B80123
:101D800086E40E9401074091AF0164E670E082E0C2
:101D900090E00E948A040FB6F894DEBF0FBECDBF5C
:101DA0009CCD8091B4019091B5019093B70180933F
:101DB000B6011092B1011092B00182E090E09093D0
:101DC000B3018093B20190939F0180939E0181E0C3
:101DD00090E09093B9018093B8010E94FA04809139
:101DE000B7018F938091B6018F938091B5018F9346
:101DF0008091B4018F9380E691E09F938F931F931E
:101E00000F930E94B517B80185E4BBCFCE018A5B62
:101E10009F4F0E944C05672B29F41092AF010E943E
:101E2000FA045BCD81E08093AF01F9CF45EAC42E7F
:101E300041E0D42E52E0E52EF12C2C968EAD9FADD4
:101E40002C97E816F90638F42896EEADFFAD2897E2
:101E5000309709F091C010927A01EAE7F1E06081D1
:101E6000C8010E943D06C70101972C962EAD3FADDB
:101E70002C978217930738F42896EEADFFAD28977C
:101E8000309709F07CC010927A01EAE7F1E06081B6
:101E9000CE018E960E943D06C70102972C962EAD6C
:101EA0003FAD2C978217930738F42896EEADFFAD1F
:101EB0002897309709F066C010927A01EAE7F1E0BE
:101EC0006081CE01CA960E943D061DAA1CAA1FAAC7
:101ED0001EAA19AE18AEBE01665C7F4FCE01C49635
:101EE0000E945506BE01625D7F4FCE01C4960E94DE
:101EF000D205B8010E94D20522961FAE1EAE2297CF
:101F000024961FAE1EAE249726961FAE1EAE2697B1
:101F1000BC01CE01805C9F4F0E945506CE01C49645
:101F20000E94A205CE01CA960E94A205CE018E96FD
:101F30000E94A205C8010E94A205CE01805C9F4FAD
:101F40000E944C0597FD21C06F3F710581059105E9
:101F500009F0F4F4F601619371936F01CE01805C96
:101F60009F4F0E94A205F3E0EF0EF11C21E1E21663
:101F7000F10409F062CF53CFEE0DFF1D70CFE80FD3
:101F8000F91F85CFE80FF91F9BCF70E060E0E2CF2B
:101F90006FEF70E0DFCFCE018A5B9F4F0E944C0550
:101FA000672B39F41092A40160E082E00E94BA012C
:101FB00036CF81E08093A40161E0F7CFCE018A5B48
:101FC0009F4F0E944C054B011092B9011092B8012D
:101FD00081E090E09093B1018093B00110929F0155
:101FE00010929E010E94FA048FE1889D7001899DE4
:101FF000F00C1124C7010E94A6038091B4019091B6
:10200000B501E80EF91EF092B501E092B4010E940C
:10201000CA041092B1011092B00182E090E0909356
:10202000B3018093B2010E94FA048091B7018F93AB
:102030008091B6018F938091B5018F938091B40107
:102040008F939F928F928CE591E09F938F931F9334
:102050000F930E94B517B8018DE44FCE80912403F1
:10206000843450F180916002909161028254910910
:102070008E9710F590E080E040E050E0BA01FC015E
:10208000EE59FD4F20813181295031092930310528
:1020900098F4FC01EC59FD4F208131812651310922
:1020A0002131310508F488C0208131812650310961
:1020B0002730310508F499C096E0291631040CF454
:1020C000EFCCA7E5B2E06496BFAFAEAF6497E3E0B4
:1020D000F0E06696FFAFEEAF669795ECC92E9DE9EE
:1020E000D92E9CE1E92E91E8F92E66968EAD9FAD32
:1020F0006697821593050CF07DC06496AEADBFADBA
:1021000064971B966D917C911C971796AD90BC902F
:1021100090E080E00E948E132B013C01B50190E01D
:1021200080E00E948E134B015C012DEC3CEC4CE4F2
:102130005FE30E94EF139B01AC01C301B2010E9457
:102140008913F0E0E0E087FD14C02DEC3CEC4CE49A
:102150005FE3C301B2010E94EF139B01AC01C50113
:10216000B4010E948913E2E0F0E087FD02C0E1E0E3
:10217000F0E0A701960163E971E080E091E00E9440
:1021800014156F01FF0FEE08FF08C626D726E826B4
:10219000F9266696EEADFFAD669731966696FFAF6F
:1021A000EEAF669764968EAD9FAD64970296649687
:1021B0009FAF8EAF649799CF440F551F661F771F4F
:1021C000416004968038910509F059CF80E290E093
:1021D0009093900180938F0140938B0150938C01D9
:1021E00060938D0170938E01C2CB440F551F661F03
:1021F000771FE7CFC0928B01D0928C01E0928D01C6
:10220000F0928E0180E290E09093900180938F0194
:102210008FEF9FEFAECB8093830190938401A093C7
:102220008501B0938601109282018CE280930001B7
:1022300040927E0150927F016092800170928101F4
:1022400010927D01C0CBE7E5CE16E8EADE06EAE9AA
:10225000EE06E6EAFE0609F499C0FDE3CF16F2ECBD
:10226000DF06FAE9EF06F6EAFF0609F40AC12DE5F2
:10227000C21622EAD2062AE9E20626EAF20609F0A6
:10228000F2CB4091AF0164E670E081E090E00E9403
:102290008A042091B8013091B9012130310591F4BF
:1022A0008091B6019091B70140919E0150919F019C
:1022B0004130510509F0DDC01092B3011092B20116
:1022C0000E9400054091AF0164E670E082E090E07A
:1022D0000E948A04C8CB4091AF0164E670E081E0BF
:1022E00090E00E948A048091A0019091A101892B25
:1022F00099F481E090E09093A1018093A0018FEF89
:102300009FEF90937C0180937B018091A20190913B
:10231000A3010E942903A9C01092A1011092A0015B
:1023200090E080E0F6CF0E947E0480907E01909045
:102330007F01A0908001B0908101AB01BC014819E0
:1023400059096A097B098091000190E0B0E0A0E0A2
:10235000481759076A077B0708F023C184CB80918F
:10236000A401811180CBFF24F394F092A40161E0D9
:1023700082E00E94BA014091AF0164E670E082E021
:1023800090E00E948A04F09299016DCB8091A001A7
:102390009091A101019709F083CBF0908201F11097
:1023A00035C00E947E0460937E0170937F0180930C
:1023B000800190938101F11045C04091AF0164E626
:1023C00070E081E090E00E948A0480917B0190910E
:1023D0007C011816190614F081E090E07C01E1E020
:1023E000EE1AF108F0927C01E0927B01E114F10415
:1023F00009F401C1F701EE0FFF1FE656FE4F83857A
:1024000094859093A3018093A20183CF0E947E04C0
:1024100080907E0190907F01A0908001B09081011A
:10242000AB01BC01481959096A097B098091000177
:1024300090E0B0E0A0E0481759076A077B0708F072
:10244000B0CF11CB8091A401882309F40CCB10925A
:10245000A40160E082E00E94BA014091AF0164E60D
:1024600070E082E090E00E948A0481E0809399010C
:10247000FACA3093B3012093B201919581959109E5
:102480001FCF8091A0019091A101019709F008CB85
:10249000B0908201BB20C9F080917E0190917F01B4
:1024A000A0918001B0918101B301A201481B590B99
:1024B0006A0B7B0B8091000190E0B0E0A0E0481730
:1024C00059076A077B0708F4D4CA40927E015092EC
:1024D0007F0160928001709281013091A201209170
:1024E000A301832F922FFDE3CF16F2ECDF06FAE96A
:1024F000EF06F6EAFF0609F58F3F910514F08EEF1F
:1025000090E001969093A3018093A2018091A20193
:102510009091A3010E94290381E080939901BB203F
:1025200009F4A1CA80910001833308F49CCA845144
:10253000823350F08093000196CA8230910514F4E2
:1025400082E090E00197DECF82E3F4CF87E6C81601
:1025500088E9D8068AE9E80686EAF80609F491CF00
:102560000CF052C0ADEFCA16A2E0DA06AAE9EA06FC
:10257000A6EAFA0609F4AFCEBDEDCB16B2E2DB0651
:10258000BAE9EB06B6EAFB0609F08ACA8091A00117
:102590009091A101019709F083CAF0908201F11096
:1025A000C2CE0E947E0460937E0170937F0180936F
:1025B000800190938101F110D2CE4091AF0164E689
:1025C00070E081E090E00E948A0480917B0190910C
:1025D0007C018430910514F083E090E07C01AFEF42
:1025E000EA1AFA0AF0927C01E0927B01B4E0EB1661
:1025F000F10409F0FFCE4091AF0164E670E082E0A3
:1026000090E00E948A04F6CEE7E5CE16E8EADE0600
:10261000EAE9EE06E6EAFE0609F4B8CEFDE3CF16D7
:10262000F2ECDF06FAE9EF06F6EAFF0609F429CF35
:102630002DE5C21622EAD2062AE9E20626EAF206C9
:1026400009F41FCE2DCACF93DF93C0912B03D091F5
:102650002C032097E1F0FE0132972081318146E082
:10266000429FC001439F900D1124C80FD91F9E01A6
:1026700080912B0390912C0326978217930721F0CA
:10268000CE010E94A205F3CF02970E942F168FE27F
:1026900093E0DF91CF910C94A2051F93FC01992741
:1026A0008827BC01E89411911032E9F3193010F039
:1026B0001E30C8F31B3251F01D3249F4689406C035
:1026C0000E947413610F711D811D911D1191105392
:1026D0001A30B0F33EF490958095709561957F4FD8
:1026E0008F4F9F4F1F910895592F482F372F262F17
:1026F000660F771F881F991F660F771F881F991F06
:10270000620F731F841F951F660F771F881F991F05
:1027100008950E94CB1308F481E00895E89409C05D
:1027200097FB3EF490958095709561957F4F8F4F04
:102730009F4F9923A9F0F92F96E9BB279395F6951A
:10274000879577956795B795F111F8CFFAF4BB0F98
:1027500011F460FF1BC06F5F7F4F8F4F9F4F16C0FC
:10276000882311F096E911C0772321F09EE8872F86
:10277000762F05C0662371F096E8862F70E060E042
:102780002AF09A95660F771F881FDAF7880F9695BB
:10279000879597F90895990F0008550FAA0BE0E85F
:1027A000FEEF16161706E807F907C0F01216130613
:1027B000E407F50798F0621B730B840B950B39F453
:1027C0000A2661F0232B242B252B21F408950A26B9
:1027D00009F4A140A6958FEF811D811D08950E94E7
:1027E00002140C9473140E94651438F00E946C1447
:1027F00020F0952311F00C945C140C9462141124B5
:102800000C94A7140E94841470F3959FC1F3950F44
:1028100050E0551F629FF001729FBB27F00DB11D64
:10282000639FAA27F00DB11DAA1F649F6627B00DF4
:10283000A11D661F829F2227B00DA11D621F739FDD
:10284000B00DA11D621F839FA00D611D221F749FEB
:102850003327A00D611D231F849F600D211D822F32
:10286000762F6A2F11249F5750409AF0F1F0882359
:102870004AF0EE0FFF1FBB1F661F771F881F915086
:102880005040A9F79E3F510580F00C945C140C94C5
:10289000A7145F3FE4F3983ED4F386957795679548
:1028A000B795F795E7959F5FC1F7FE2B880F911DB0
:1028B0009695879597F9089597F99F6780E870E056
:1028C00060E008959FEF80EC089500240A941616A6
:1028D000170618060906089500240A94121613060E
:1028E000140605060895092E0394000C11F488239C
:1028F00052F0BB0F40F4BF2B11F460FF04C06F5FB8
:102900007F4F8F4F9F4F089557FD9058440F551F8D
:1029100059F05F3F71F04795880F97FB991F61F061
:102920009F3F79F087950895121613061406551FD8
:10293000F2CF4695F1DF08C0161617061806991F44
:10294000F1CF86957105610508940895E894BB2739
:1029500066277727CB0197F90895F999FECF92BDA5
:1029600081BDF89A992780B50895262FF999FECF51
:102970001FBA92BD81BD20BD0FB6F894FA9AF99A9C
:102980000FBE019608950E940515A59F900DB49F56
:10299000900DA49F800D911D112408952F923F92B8
:1029A0004F925F926F927F928F929F92AF92BF925F
:1029B000CF92DF92EF92FF920F931F93CF93DF930B
:1029C000CDB7DEB7CA1BDB0B0FB6F894DEBF0FBE68
:1029D000CDBF09942A88398848885F846E847D84B5
:1029E0008C849B84AA84B984C884DF80EE80FD80B7
:1029F0000C811B81AA81B981CE0FD11D0FB6F8942D
:102A0000DEBF0FBECDBFED010895A29FB001B39F01
:102A1000C001A39F700D811D1124911DB29F700DE7
:102A2000811D1124911D0895DB018F939F930E94B6
:102A3000C314BF91AF91A29F800D911DA39F900DD4
:102A4000B29F900D1124089597FB072E16F4009461
:102A500007D077FD09D00E945D1507FC05D03EF434
:102A6000909581959F4F0895709561957F4F08953A
:102A7000052E97FB1EF400940E944F1557FD07D0BA
:102A80000E94711507FC03D04EF40C944F1550951D
:102A90004095309521953F4F4F4F5F4F089590954A
:102AA0008095709561957F4F8F4F9F4F0895EE0FE2
:102AB000FF1F0590F491E02D0994AA1BBB1B51E167
:102AC00007C0AA1FBB1FA617B70710F0A61BB70B9E
:102AD000881F991F5A95A9F780959095BC01CD0143
:102AE0000895A1E21A2EAA1BBB1BFD010DC0AA1F4F
:102AF000BB1FEE1FFF1FA217B307E407F50720F067
:102B0000A21BB30BE40BF50B661F771F881F991FE1
:102B10001A9469F760957095809590959B01AC012A
:102B2000BD01CF0108950F931F93CF93DF938230A0
:102B3000910510F482E090E0E0915103F09152038E
:102B400030E020E0B0E0A0E0309799F421153105A5
:102B500009F44AC0281B390B24303105D8F58A8185
:102B60009B816115710589F1FB0193838283FE01CD
:102B700011C0408151810281138148175907E0F04B
:102B80004817590799F4109761F012960C93129711
:102B900013961C933296CF01DF91CF911F910F9125
:102BA00008950093510310935203F4CF211531057A
:102BB00051F04217530738F0A901DB019A01BD011A
:102BC000DF01F801C1CFEF01F9CF90935203809359
:102BD0005103CDCFFE01E20FF31F81939193225059
:102BE000310939832883D7CF20914F033091500387
:102BF000232B41F4209103013091040130935003C1
:102C000020934F03209101013091020121153105DC
:102C100041F42DB73EB74091050150910601241BA8
:102C2000350BE0914F03F0915003E217F307A0F446
:102C30002E1B3F0B2817390778F0AC014E5F5F4F12
:102C40002417350748F04E0F5F1F509350034093F1
:102C50004F03819391939FCFF0E0E0E09CCFCF931F
:102C6000DF930097E9F0FC01329713821282A09162
:102C70005103B0915203ED0130E020E01097A1F430
:102C800020813181820F931F20914F033091500397
:102C90002817390709F061C0F0935003E0934F0300
:102CA000DF91CF910895EA01CE17DF07E8F54A8159
:102CB0005B819E0141155105B1F7E901FB83EA8370
:102CC00049915991C40FD51FEC17FD0761F480811C
:102CD00091810296840F951FE901998388838281EF
:102CE00093819B838A83F0E0E0E012968D919C9122
:102CF00013970097B9F52D913C911197CD0102964C
:102D0000820F931F20914F033091500328173907EA
:102D100039F6309751F51092520310925103B09347
:102D20005003A0934F03BCCFD383C2834081518112
:102D3000840F951FC817D90761F44E5F5F4F8881D4
:102D40009981480F591F518340838A819B819383C6
:102D500082832115310509F0B0CFF0935203E0933F
:102D600051039ECFFD01DC01C0CF13821282D7CF69
:102D7000B0E0A0E0EEEBF6E10C94D0148C010097EB
:102D800051F4CB010E9493158C01C801CDB7DEB779
:102D9000E0E10C94EC14FC01E60FF71F9C012250BB
:102DA0003109E217F30708F49DC0D901CD91DC91F8
:102DB0001197C617D70798F0C530D10530F3CE016B
:102DC00004978617970708F3C61BD70B2297C19362
:102DD000D1936D937C93CF010E942F16D6CF5B01C8
:102DE000AC1ABD0A4C018C0E9D1EA0915103B091EE
:102DF0005203512C412CF12CE12C109731F580918C
:102E00004F03909150038815990509F05CC0461650
:102E1000570608F058C08091010190910201009777
:102E200041F48DB79EB74091050150910601841B76
:102E3000950BE817F90708F055C0F0935003E0939D
:102E40004F03F90171836083A0CF8D919C911197FD
:102E500012966C90129713967C901397A815B9054B
:102E600059F56C0142E0C40ED11CCA14DB0420F1F8
:102E7000AC014A195B09DA011296159780F062825B
:102E8000738251834083D9016D937C93E114F104E3
:102E900071F0D7011396FC93EE93129776CF22969A
:102EA0008C0F9D1FF90191838083F301EFCFF09385
:102EB0005203E093510369CF4816590608F42C01D8
:102EC0007D01D3019ACFCB010E9493157C0100971D
:102ED00049F0AE01B8010E947517C8010E942F1673
:102EE000870153CF10E000E050CFFB01DC0102C0AE
:102EF00001900D9241505040D8F70895FB01DC013C
:102F000001900D920020E1F70895AEE0B0E0EBE80B
:102F1000F7E10C94DC140D891E898F89988D26E0C9
:102F20002C831A83098397FF02C080E090E8019701
:102F30009E838D83AE01455E5F4F698D7A8DCE0194
:102F400001960E94D8174D815E8157FD0AC02F81DE
:102F50003885421753070CF49A01020F131FF8012A
:102F600010822E96E4E00C94F814AEE0B0E0EBEBA7
:102F7000F7E10C94DC140D891E8986E08C831A839A
:102F800009838FEF9FE79E838D83AE01475E5F4F7E
:102F90006F89788DCE0101960E94D8172F813885D0
:102FA000020F131FF80110822E96E4E00C94F8141F
:102FB000ABE0B0E0EEEDF7E10C94CE147C013B0108
:102FC0008A01FC0117821682838181FFC8C1CE016C
:102FD00001965C01F7019381F30193FD859193FFC5
:102FE00081913F01882309F453C1853239F493FD5F
:102FF000859193FF81913F01853229F4B70190E0DB
:103000000E94C819E7CF912C212C312CFFE1F31538
:1030100038F08B3211F190F4803209F1833229F1CA
:1030200037FC3CC020ED280F2A3050F536FE20C07A
:103030008AE0989E200D1124922E06C08D3291F0C8
:10304000803371F7689430F8F30193FD859193FF15
:1030500081913F018111DACF21C0689431F86894E1
:1030600032F8F2CF689433F8EFCF689434F8ECCFAD
:10307000EAE02E9E200D1124222E689435F8E4CF2C
:103080008E3229F436FC04C1689436F8DDCF8C36D4
:1030900019F4689437F8D8CF8836B1F2982F9F7D0D
:1030A00095549330E0F08336A1F18337C1F1833535
:1030B00009F063C02801F2E04F0E511CF801C080F6
:1030C000D180692D70E036FC02C06FEF7FEFC60142
:1030D0000E94B2194C01689437F882010AC00C5F53
:1030E0001F4FFFE3F98388248394912C6501E894B2
:1030F00037F833FE2DC0522C8114910471F5552000
:1031000009F468CFB70180E290E00E94C8195A9490
:10311000F6CFF801808189830E5F1F4FE4CF28012D
:10312000F2E04F0E511CF801C080D180692D70E093
:1031300036FC02C06FEF7FEFC6010E94BD194C0143
:103140008201D5CFB70180E290E00E94C8192A948D
:103150002814190409F0B0F7CECFF60137FC859199
:1031600037FE81916F01B70190E00E94C81951109C
:103170005A94F1E08F1A9108BFCF843619F089363E
:1031800009F077C0F80137FE6BC0608171818281E0
:1031900093810C5F1F4FF32DFF763F2E97FF09C0E1
:1031A00090958095709561957F4F8F4F9F4F689454
:1031B00037F82AE030E0A5010E94F819C82ECA1895
:1031C0008C2C432C36FE0CC0E89440F8C91440F413
:1031D00034FE05C032FC03C0F32DFE7E4F2E892C39
:1031E00044FE95C0FE01EC0DF11D8081803309F095
:1031F00087C0242D297E422E842D8870582E43FCB2
:1032000095C040FE8FC09C2C821418F42C0C922C7C
:10321000981844FE91C0B70180E390E00E94C8195D
:1032200042FE09C088E790E041FE02C088E590E0D8
:10323000B7010E94C819C91408F48AC0CA94D12CD5
:103240009FEFC91AD90ACA0CDB1CF60182916F01E3
:10325000B70190E00E94C819AC14BD04B1F74FCF7C
:1032600060817181072E000C880B990B0E5F1F4F38
:1032700092CFD32CE894D4F82AE030E0853739F1A6
:10328000232D297FD22E8F3601F148F48835A9F0FD
:10329000F701868197812B96E2E10C94EA1480373E
:1032A00049F08837A9F7D4FE02C06894D2F820E12B
:1032B00030E00DC06894D4F8F6CF34FE03C0822FFE
:1032C0008660D82E20E132E002C028E030E0F8012C
:1032D000D7FE0FC060817181828193810C5F1F4F87
:1032E000A5010E94F819C82ECA183D2CE89437F899
:1032F00067CF6081718190E080E00E5F1F4FF0CF5B
:1033000042FC02C0839478CF8394839475CF842D3C
:10331000867809F471CFF6CFB70180E290E00E9481
:10332000C81983948214C0F3512C73CF522C5818AF
:10333000821408F46ECFF8CF842D867809F47BCF01
:103340008BE241FE80E247FC8DE2B70190E071CF55
:10335000B70180E390E00E94C8199A946CCF8FEF78
:103360009FEF99CFFC010590615070400110D8F794
:10337000809590958E0F9F1F0895FC0161507040BD
:1033800001900110D8F7809590958E0F9F1F08959A
:103390000F931F93CF93DF93182F092FEB018B818E
:1033A00081FD09C01FEF0FEF812F902FDF91CF918B
:1033B0001F910F91089582FF14C02E813F818C814F
:1033C0009D81281739073CF4E881F981CF010196E6
:1033D0009983888310838E819F8101969F838E833A
:1033E000E3CFE885F985812F0995892BA1F3DACF01
:1033F000FA01AA27283051F1203181F1E8946F9326
:103400006E7F6E5F7F4F8F4F9F4FAF4FB1E03ED0CB
:10341000B4E03CD0670F781F891F9A1FA11D680F69
:10342000791F8A1F911DA11D6A0F711D811D911D9C
:10343000A11D20D009F468943F912AE0269F112411
:103440003019305D3193DEF6CF010895462F477075
:10345000405D4193B3E00FD0C9F7F6CF462F4F70D0
:10346000405D4A3318F0495D31FD4052419302D02E
:10347000A9F7EACFB4E0A6959795879577956795D4
:10348000BA95C9F700976105710508959B01AC01D4
:103490000A2E06945795479537952795BA95C9F7FB
:1034A000620F731F841F951FA01D089510E0C2E6D0
:1034B000D0E004C0FE010E9457152196C336D10703
:0634C000C9F7F894FFCFEC
:1034C6002C0000530380003430380047656D696E68
:1034D60069466C617450616E656C000000000024E2
:1034E600018E00BB007101EC00CA00DE002A2563D4
:1034F60025732563002A256325642563004F7065BF
:103506006E656400436C6F736564002564256425ED
:1035160064256400256452656164790053742564EA
:0A352600436125644F612564000035
:00000001FF
